:10000000F3C0FECF3AC1FCCFFBCFFACF2BC2F8CF63
:10001000F7CF68C1F5CFF4CFF3CFF2CFF1CFF0CF68
:10002000EFCFEECFEDCF040506050000000000196C
:1000300012140B120300000000001B151500040E23
:100040001F00040E0400000E00001F0E04000C121E
:100050000C00000000001F111D1117111F000000EF
:100060000000000000006400C80090012003F8FFB9
:10007000FCFFFEFFFFFF000000000000001E01006B
:1000800063322E61742E756100706F726F67006F3E
:10009000622F6D004D4D4D65747256490020002E43
:1000A000005600010203003939393900393939392C
:1000B0003900487A00202D002E3006430020202DE4
:1000C00000202B00202020300020202B00BE6FB805
:1000D00063BA20445300766F6C746D65747200745B
:1000E00061786F6D657472006461766C656E6965C8
:1000F000004D4D4D2D6D657472007465726D6F2DE0
:100100007472000405206E6578743E0020563D0030
:100110002004053E006176742E43406174006B6FCD
:10012000656666692D20006369656E743D00346103
:1001300073746F746F2D006D657220487A0405002A
:1001400020463D00487A200020443D00205665723C
:100150005F492E3000696E7665727369610076784A
:100160006F6420002044410048455400746F636868
:100170006B6100302E30003030006D616B732E20CB
:10018000646F006F737461742E0062756B76613DED
:100190000006433D005465726D6F6D2D2000747232
:1001A0003E0020564B4C3C004F544B4C3C00767567
:1001B000686F6420697A006D656E6A7520203E0064
:1001C00080C0010002007600090060018000060086
:1001D0006901890005006F018F00080004007800A4
:1001E0000200AE01C0010000F894EE27ECBBF1E084
:1001F000FBBFEBBFE5BFF8E1F1BDE1BD8DE0A2E0E3
:10020000BB27ED938A95E9F780E094E0A0E6ED93B3
:100210000197E9F7E2ECF1E085919591009761F0A3
:10022000A591B59105901590BF01F00105900D9233
:100230000197E1F7FB01F0CFEFE5EDBFE4E0EEBFA2
:10024000C0E6D1E0F9C2AA9353DEEA81EE0FEE0FC9
:10025000EE0FE0640E2F10E0183060F40A9303955F
:10026000EC81FD813196EC83FD833197A491E7D732
:100270001F5FF2CF42DE259608956A937A938A93A0
:10028000AA93BA93EA93FA93EFB7EA93A6E8B1E098
:10029000CCDDEF5FFF4F6F4F7F4FCCDD89D820F073
:1002A00083E48A95F1F703C08DE08A95F1F7E9912F
:1002B000EFBFF991E991B991A991899179916991EA
:1002C0001895AA93E881E064E7B98BE18A95F1F784
:1002D000369A349BFECF349AE4B1F5B1662777277E
:1002E000219608950A921A92FA926A937A938A93BF
:1002F0009A93AA93BA93EA93FA93EFB7EA93A895DD
:10030000EFE7E2BFE62D6394E91508F44FC06624D9
:1003100054D856D85ED8E0939E01F0939F01609325
:10032000A0017093A10149D857D853D8E093A201F6
:10033000F093A3016093A4017093A5013ED855D812
:1003400048D8E093A601F093A7016093A8017093A9
:10035000A90133D853D83DD8E093AA01F093AB015B
:100360006093AC017093AD01E0E0E0938E01E09307
:100370008F01E0939001E0939101E0939201E0936B
:100380009301E0939401E0939501E0939601E0934B
:100390009701E0939801E0939901E0939A01E0932B
:1003A0009B01E0939C01E0939D014EC0A0E089DF9A
:1003B00007D89EDCE0938E01F0938F01609390014B
:1003C00070939101A1E07DDFA3E0B0E080E090E0D8
:1003D000AFDC02D88DDCE0939201F093930160933F
:1003E000940170939501A2E012D8FFD781DCE093CD
:1003F0009601F093970160939801709399010FD83B
:10040000E13061F4A3E05DDF7F936F93FF93EF939F
:100410000AD8AF91BF918F919F910BC0A3E0F7D7FE
:100420007F936F93FF93EF93FED7AF91BF918F911F
:100430009F917EDCE3D75CDCE0939A01F0939B0113
:1004400060939C0170939D01E991EFBFF991E9914F
:10045000B991A9919991899179916991F99019909E
:10046000099018950A921A926A937A938A939A93AA
:10047000AA93BA93EA93FA93EFB7EA93D8D7E5E051
:10048000E51501F595D790F0D6D7ACE3B0E080E064
:1004900090E04EDC7F936F93FF93EF93D5D7D8D73F
:1004A000AF91BF918F919F9194D701C0C4D7E09332
:1004B0008A01F0938B0160938C0170938D01689495
:1004C00024F85524539424FE0BC0E0E0E093860109
:1004D000E0938701E0938801E0938901E89424F890
:1004E000E1E08E1608F0B39421FE02C0439401C0EF
:1004F0004424E991EFBFF991E991B991A9919991BA
:10050000899179916991199009901895882021F520
:10051000A1D721F4B19B02C0B29901C006C0B09B23
:10052000FECF9DD79FD79BD7A0D7B09B04C0B19BD0
:1005300002C0A0D709F006C0B29BFECFA0D792D7C9
:100540009ED793D79FD7E43010F089D79ED7A0D7F6
:10055000E43010F094D799D7B09B07C0A0E0B199D0
:10056000A1E0A03011F4B29901C006C0B19BFECF4A
:100570008394BB2490D78DD6E1E08E1628F06AD7FD
:1005800011F078D709F4BB24E1E0E815C9F4B0997B
:100590000AC0B09BFECF82D765D783D7E53010F075
:1005A0007DD773D783D7B2990BC0B29BFECF81D7CB
:1005B000E15077D7E63018F071D7E4E078DC76D7F1
:1005C000E2E08E1608F437C174D7E03011F474D726
:1005D00009F016C0B09907C072D774D779D710F058
:1005E0006ED782D787D7B2990BC087D789D770D7F4
:1005F00030F065D7E2ECFBE060E070E048DC7AD7F1
:1006000058D7E130D9F458D7C9F4B0990AC01CD7EB
:10061000EF5F7BD74CDC18D7E13110F076D735D7B8
:1006200077D7B2990BC010D7E1506FD740DC0CD709
:10063000E13118F06AD7E0E13ADC6AD76CD729F5E6
:10064000B09912C06BD70FDCEB5FFF4F6F4F7F4F3E
:1006500068D7EC30A7E2FA07A0E06A07A0E07A07C3
:1006600010F05CD741D722D7B2990FC05FD7E550C1
:10067000F0406040704055D72BDC31F44FD7EBE0B1
:10068000F7E260E070E003DC11D713D7E23011F439
:1006900013D709F016C0B09907C04BD713D74CD762
:1006A00010F047D721D726D7B2990BC051D728D7FA
:1006B00043D730F03ED7E2EFF3E060E070E0E7DBF5
:1006C00019D7F7D6E33009F08EC0F6D681F4C2D63A
:1006D00011F0D0D661F4A3D6EF5FA5E0B0E0E7DB80
:1006E0009ED6E23018F0A5E0B0E0CFD611D713D7F0
:1006F00071F4B0D611F0BED651F42DD7B3D62BD7A6
:10070000D6DB2CD7E23010F026D7BFD601D729D7B9
:1007100031F5B09911C087D6EF5FFF4F6F4F7F4F14
:1007200023D7B5DB80D623D730F01ED7E1E0F0E049
:1007300060E070E0ACDBECD6B29911C074D6E15049
:10074000F0406040704010D7A2DB6DD6C1DB31F4C1
:100750000BD7E9E0F0E060E070E099DBD9D6E5E0A6
:10076000E81551F5B09912C00AD7ACD60BD77F93D4
:100770006F93FF93EF9357D60AD7AF91BF918F91A5
:100780009F91AADB10F4FBD6AFD685D6B29914C0E0
:1007900004D7B6D6F7D67F936F93FF93EF9343D6E4
:1007A000F6D6AF91BF918F919F9196DB20F43BD607
:1007B000EED6E5D66CDB6FD6E6E0E815A1F4B0998D
:1007C00008C0EED64FD6EFD618F4EAD6E1E26FDBDA
:1007D00091D6B29908C0EDD6E150E5D618F4E0D62E
:1007E000EEEF65DB87D665D6E43029F565D699F45A
:1007F000B09907C0E1D636D6E2D610F0DDD645D6A0
:1008000079D6B29908C0E1D6E150D9D618F0D4D63D
:10081000EDE74DDB6FD67FD671F41CD611F02AD6EA
:1008200051F4D6D61FD6D4D642DBD5D6E23010F05E
:10083000CFD62BD66DD60895E7E0E8BBE0E3E7BB63
:10084000E0ECE5BBE1E3E4BBE8E0E2BBE0E0E1BB18
:10085000E5E0E3BFE0E0E2BFEFBDE5E0EEBDE7D5F8
:10086000E0E0E7BDE6BDE6E0EBBDEAE1EABDE0E0E1
:10087000E9BDE8BDE2BDE5BDE4BDE3BDEBB7E068C1
:10088000EBBFECE0E5BFE0E8EABFE1E1E9BFE0E8AB
:10089000E8B9E0E0E0BFE0ECE7B9E3E8E6B9A8E0FA
:1008A0005AD5E0EFEA93ADE7B1E0BBD8AE2E88248D
:1008B00095D697D699D6D8011FD593D697D6A4E9C1
:1008C000B0E027D5A0E2B3E052D8E6E2F0E090D65F
:1008D000A1E0B9DCEEE2F0E08BD6A2E0B4DCE6E326
:1008E000F0E086D6A3E0AFDCEEE3F0E081D6A4E052
:1008F000AADCE6E4F0E07CD6A5E0A5DCEEE4F0E0DE
:1009000077D6A6E0A0DCE6E5F0E072D6A7E09BDCB7
:10091000EEE5F0E06DD6A8E096DCBBD47894F6DD89
:10092000882009F042C15DD65FD6ACD5E03049F4ED
:1009300062D664D66CD610F4A0E201C070D6B8D4EA
:100940007ED6A0D5E130C1F456D69FD660D610F43D
:10095000A0E201C0A3D6ACD4B1D618F4FFD5E130E3
:1009600009F002C0A0E201C0B2D6A2D4F7D5E030AF
:1009700009F4BDD6BFD6CFD685D5E23071F43BD6CB
:10098000CCD645D610F4A0E201C0D0D691D4DED6A4
:10099000AED6EBD6A3EAB0E0BCD474D5E330B9F55B
:1009A000F3D6FBD610F004D508F404C0A7EAB0E0F3
:1009B000B0D425C0FAD620F0ACEAB0E0AAD41FC06B
:1009C00043D5E03031F4FAD610F4A0E201C0FFD6EE
:1009D0006FD4DAD61CD610F4A0E201C008D768D4D0
:1009E00016D710F4A0E201C01BD762D429D710F4A7
:1009F000A0E202C02ED733D75BD42BD73BD7D8D4B5
:100A000018F0DA0179D403C0A2EBB0E082D4E9D5C2
:100A1000EDD53ED5E03049F4EED5F0D5F8D510F45B
:100A2000A0E201C0FCD544D40AD632D5E130C1F4ED
:100A3000E2D52BD6ECD510F4A0E201C02FD638D4E5
:100A40003DD618F48BD5E13009F002C0A0E201C018
:100A50003ED62ED483D5E03009F449D64BD65BD6AA
:100A600017D5E23071F4C7D558D6D1D510F4A0E22D
:100A700001C05CD61DD46AD63AD677D6A3EAB0E0D8
:100A800048D406D5E33009F090C0A5D5E03009F090
:100A900055C022FC32C020FC1BC0EAEAFFE0CE16A3
:100AA000DF0634F0A5EBB0E0E8D6ECD6F2D6F7D608
:100AB000E0EAFFE0CE16DF0624F0E9EAFFE0F2D636
:100AC0000CF405C0ADEBB0E0D8D6EFD6E8D615C033
:100AD00023FE05C0A1ECB0E0D0D6D4D6DAD623FCF4
:100AE0000BC0A2ECB0E015D4D601E4E6F0E0CAD623
:100AF000D601DED6C7D6CDD6D2D622FE16C0A0E00D
:100B000020FCA1E0A03011F4D6D609F004C0A4EC7A
:100B1000B0E0FFD3C4D620FE02C0CDD609F005C098
:100B2000A9ECB0E0AAD6C1D6BAD6EEE34E1628F0AC
:100B300058D55CD5ADECB0E0ECD337C025D62DD67A
:100B400010F036D408F404C0A7EAB0E0E2D325C020
:100B50002CD620F0ACEAB0E0DCD31FC075D4E03076
:100B600031F42CD610F4A0E201C031D6A1D30CD6BA
:100B70004ED510F4A0E201C03AD69AD348D610F46C
:100B8000A0E201C04DD694D35BD610F4A0E202C01F
:100B900060D665D68DD35DD66DD60AD418F0DA014D
:100BA000ABD303C0A2EBB0E0B4D3E1E08E1608F4FF
:100BB000B9C1E81529F515D517D57BD4E03019F45E
:100BC000A6EDB0E0A6D375D4E13019F4AFEDB0E0F6
:100BD000A0D36FD4E23019F4A8EEB0E09AD369D470
:100BE000E33019F4A1EFB0E094D363D4E43019F406
:100BF000AAEFB0E08ED3F5D4F9D4A3E0B1E089D365
:100C000058D4E03041F558D4C1F4EBD4EDD458D6E3
:100C1000ACE0B1E057D6EAD470D456D610F4A0E2D6
:100C200003C06BD459D65BD643D367D45DD662D6A6
:100C30005ED563D466D65ED66AD66DD449F4D1D477
:100C4000D3D4D80159D3CDD4D1D4A5E1B1E061D367
:100C500088D409F45FD62DD4E13009F04FC02CD4EC
:100C6000D9F4BFD4C1D4A4D380F0AEE1B1E02AD688
:100C7000BDD4A7E2B1E04DD3E7D34FD68CD8E05D29
:100C80004AD5E2D34AD611D607C0AEE2B1E01AD6B1
:100C9000ADD4A7E3B1E03DD33ED469F5A2D4A4D44A
:100CA0000FD6A0E4B1E00ED6A1D440D40DD610F4F6
:100CB000A0E203C03BD410D612D6FAD237D430D635
:100CC00010F4A0E203C032D40FD6C9D5F1D22ED48D
:100CD0004ED410F4A0E203C029D413D6C0D5E8D274
:100CE00025D40FD6C7D564D318F0DA0105D303C0D5
:100CF000A4E4B1E00ED335D409F40CD6DAD3E23053
:100D000041F5DAD3C1F46DD46FD4DAD5A8E4B1E0FB
:100D1000D9D56CD41DD4D8D510F4A0E203C018D412
:100D2000DBD5DDD5C5D214D4DFD5E4D5E0D410D4DD
:100D3000E8D5E0D5ECD5EFD349F453D455D4A1EFA1
:100D4000B0E0C0D553D4ACE4B1E0E3D20AD409F4A6
:100D5000E1D5AFD3E33009F096C0AED391F441D4DE
:100D600043D4A5E5B1E0AED541D4AEE5B1E0D1D2F2
:100D700056D3E03019F4A4E6B1E002C0A8E6B1E031
:100D8000C8D2C9D3C1F42DD42FD4ACE6B1E09AD5E2
:100D90002DD4CED5B6D56ED5E1D3E03019F4A3E786
:100DA000B1E002C0A7E7B1E0B4D203D4B4D4D6D343
:100DB000E13009F420D4D5D3A1F413D415D4AAE793
:100DC000B1E080D513D4B4D59CD554D5C7D3E03089
:100DD00019F4A3E7B1E002C0A7E7B1E09AD2E9D3E2
:100DE0009AD4E5E0E81549F5FCD3FED3A3E8B1E0D9
:100DF00090D2DFD390D4AEE0B1E064D5F7D3CDD3B9
:100E000063D510F4A0E203C0C8D366D568D550D22C
:100E1000C4D386D518F4A2D3E13009F002C0A0E211
:100E200003C0BBD361D51BD543D298D3E03009F4BE
:100E30005ED4B3D366D55ED56AD5E6E0E815F9F49D
:100E4000D0D3D2D3AAE8B1E064D2B3D364D4C9D3A7
:100E5000CDD3D1D3E8D255D50DD580D3E03019F418
:100E6000A3E7B1E002C0A7E7B1E053D2A2D353D4C5
:100E700075D3E13009F4BFD3AAE0B1E04AD2E7E08C
:100E8000E81509F447D515D3E430E1F515D319F584
:100E9000A8D3AAD315D5A1E9B1E014D5A7D3A2EC64
:100EA000B0E037D292D3E43610F4A0E206C08DD37E
:100EB000CFD2DF01E4E6F0E03FD5FAD186D3EA30C5
:100EC00010F4A0E203C081D328D536D5F1D17DD36B
:100ED00024D5EBD4E4D41FD391F483D385D3A5E9EF
:100EE000B1E0F0D483D3AEE9B1E013D274D3E030F3
:100EF00019F4A2EAB1E002C0A8EAB1E00AD231D303
:100F000009F408D5E8E0E81549F46BD36DD3AEEAEF
:100F1000B1E0D8D46BD3A7EBB1E0FBD1E9E0E815A1
:100F200009F48824EAD2DF01CB01E091A201F0911B
:100F3000A3016091A4017091A501D3D710F0A898E6
:100F400001C0A89A05D3DF01CB01E091A601F09181
:100F5000A7016091A8017091A901BED710F0C498B3
:100F600001C0C49AE3D2DF01CB01E0918A01F09184
:100F70008B0160918C0170918D01B3D710F0C598F1
:100F800001C0C59A0AD3DF01CB01E091AA01F0911B
:100F9000AB016091AC017091AD01A3D710F0AC9A98
:100FA00001C0AC9821FC17C010D3AE2FF601B0E001
:100FB000AE17BF077CF46CD2E33011F420FC01C003
:100FC00009C009D3E13009F4AD9805D3E03009F444
:100FD000AD9A01C0AD98ECE34E1618F459D2E33047
:100FE00009F0AD98E2E8BE1618F053D1BB2488246E
:100FF000A0E0B0E040D7E53008F43FC040D2E3E0E5
:1010000056D72DD2E4E053D749D2E1E050D77DD274
:10101000E2E04DD7DDD2E1E04AD7E0D2A5E0B0E092
:1010200034D2A2D2E4E0F0E060E070E030D793D2B6
:101030002CD2B6D2ECE43BD7BFD2E7E138D7CED240
:101040003ED2ECEDF5E060E070E021D772D2E0E551
:10105000F0E060E070E01BD761D2E0E7F7E160E02C
:1010600070E015D78CD2E4E6F0E060E070E00FD7D6
:10107000B5D2A0E0B0E009D20ED2E5E07E1630F0A5
:10108000AAD2E03019F404D2E33009F035C0ADE75C
:10109000B1E073D07AD56F01E1E0F0E0CE16DF0663
:1010A00014F0689401C0E89420F80024C014D0041F
:1010B00024F4E4ECFFEFF6D30CF005C0E0EAFFE027
:1010C000EC19FD096F01E9E0F0E0ECD314F068944D
:1010D00001C0E89422F8E3E6F0E0E4D314F0689469
:1010E00001C0E89423F8EAEBFFEFDCD314F0689436
:1010F00001C0E89421F87724739411CCFFCF23D456
:101100001A933FD4E03011F4E0E012C1E981FA8192
:10111000309769F0A5E57BD410E018D4ED91A98350
:10112000BA83AE2F74D41F5F1830B8F302C0ACEC92
:101130006ED4E1E0FDC007D4D9D6AC81BD81DFDF3C
:10114000E03011F4E0E016C0AEEB61D410E024E72B
:1011500031E03F932F932F5F3F4F54D4AF91BF9116
:10116000EC931F5F1930A8F3E4E7F1E041D2A9E066
:10117000C7D4D9D5C0D626960895E5D31A93E6D319
:10118000DADFE03011F4E5D3D3C0E0917801E295E5
:10119000EF70E695E3701E2FD9D3B1DFE03011F484
:1011A000D8D3C6C0A4E433D4E12FA6E6B0E0D6D3AA
:1011B0004AD6DDD3CBD3BFDFE03011F4CAD3B8C0F9
:1011C000E0D3E12FAEE6B0E0C9D339D6A0917401E7
:1011D000B0917501EA23FB23A1D50ED5A0E0B0E0C4
:1011E00080E89DE337D5A4C0FFE0FA95F1F70895B4
:1011F000A1B3AF70A1BB919A9098F6DF929AF4DFF9
:10120000A0B39298F1DF929AEFDF9298A7FDF5CF05
:101210000895A07FAB2BA2BB929AE6DF9298E4DF01
:101220000895AA939198A1B3A76FA1BBB2B3BF7061
:10123000A881EFDFA881A295ECDF919AB7C0AA93AD
:10124000D7DFA981EEDFD4DF909AA881EADF1FC043
:10125000929ACADFE0B39298C7DFE07F0895C4DFB7
:10126000F7DFAE2FF5DF9198E295EA2B0895AA9368
:10127000BFDFE881EDD0E255FE4FE081A981AE0FDE
:10128000D0DFE981E093B201E881E093B3012296D7
:101290000895AEDFA2E0C5DFABDFACE0C2DFA8DFC0
:1012A000A1E0BFDFE0E0E093B301E093B201089575
:1012B000AA93EF93FF93A8816894AA3039F0E89439
:1012C000E091B401A091B201AE1750F0E091B301EA
:1012D000EF5FE093B30185D1A091B301C8DF4EF079
:1012E000E091B201EF5FE093B20182DF909AA881B2
:1012F00098DFFF91EF915AC026D31A9327D3ED912F
:10130000A983BA831E2FE03019F0A12FD1DFF6CFC9
:101310000FC019D31A93E981FA813196E983FA83D0
:101320003197E4911E2FE03019F0A12FC1DFF3CFE8
:10133000188123960895AA27BB271197F1F70895DE
:10134000AA939198A1B3A76FA1BBB2B3BF70A881B4
:1013500060DF919A2BC0AA9392989098E881E093CD
:10136000B401E058E093B001E881E054E093B101AA
:10137000FBD2FAD2F9D2DFDFA0E2E2DFDCDFA8E2C3
:1013800050DFD9DFA4E04DDFD6DFA5E84ADFD3DFA9
:10139000A1B3AF70A1BB919A62DFE53011F0E0E03C
:1013A00005C026DFA6E03DDF74DFE1E02196089569
:1013B000A4E0B0E060D5E1300895E92DF0E00895B3
:1013C000A0918E01B0918F01809190019091910137
:1013D0000895A4D4E5D40895A0919201B091930109
:1013E00080919401909195010895A0919601B091FA
:1013F000970180919801909199010895A0919A0187
:10140000B0919B0180919C0190919D01089559D7C5
:10141000AFEFB3E080E090E019D56FD40895A5E078
:10142000B0E029D50895A6E1B0E01DD50895E0E02B
:10143000EDBDECBD0895E0918601F09187016091CA
:101440008801709189010895A4E0B0E014D5089551
:10145000F0E00895A0E0B099A1E0A0300895A2E0E6
:10146000B0E0089508D5EF5F089521D5A6E9B0E072
:101470007ED20FCFA0E0B299A1E0A0300895A1E004
:10148000B0E00895ECDFF7D40895E0E010D50895BA
:10149000F6DFF1D40895A2E3B0E069C2A3E0B0E0C2
:1014A0000895FCDF04D5FADFE6D40895A6E9B0E09C
:1014B0005EC2F4DFE0D40895E2E0E8150895AAE002
:1014C000B0E00895D0D4E65FFF4F6F4F7F4F08958F
:1014D000F6DFDDD4F4DFC7D4E33CABE0FA07A0E0ED
:1014E0006A07A0E07A070895EAE0F0E060E070E0C3
:1014F000CED40895AAEFB0E03AC2E1DFB4D40895A3
:10150000EA50F040604070400895A4E0B0E00895D3
:10151000AEE5B1E02CC2E3E0E8150895A2E1B0E049
:101520000895FCDFB4D4FADF9ED40895F7DF9BD48E
:101530000895AEE0B0E00895FCDFA9D4FADF93D4BB
:10154000E33FA3E0FA07A0E06A07A0E07A07089566
:10155000F0DF89D40895A6E0B0E00895FCDF8BD4D5
:101560000895E4E0E8150895A6E1B0E00895EA30B2
:10157000A0E0FA07A0E06A07A0E07A070895AAE1D0
:10158000B0E00895FCDF83D4FADF6DD40895A8EEAF
:10159000B3E080E090E0CCD30895F1DF64D4089507
:1015A000A7E0B0E00895FCDF82D4FADF64D4E03233
:1015B0000895F6DF60D40895A8E0B0E00895FCDF58
:1015C00076D4FADF58D4EE370895F6DF54D4089570
:1015D000A9E0B0E00895FCDF4ED40895A5E0B0E0A6
:1015E000C6C1E0E0EA930895A0E041CEA1E03FCE7D
:1015F000FA93EA930895ADE9B0E08BCEA091A201F1
:10160000B091A3018091A4019091A5010895A83EF5
:10161000E3E0BE07E0E08E07E0E09E070895EEDF1E
:10162000E8EEF3E060E070E0BBD3DF01CB01EAE07D
:10163000F0E060E070E0E7D3E05DAE2F0895DEDF1C
:10164000E4E6F0E060E070E0ABD3DF01CB01EAE07C
:10165000F0E060E070E0D7D3E05DAE2F29DEAFE9C7
:10166000B0E057DECBDFEAE0F0E060E070E098D376
:10167000DF01CB01EAE0F0E060E070E0C4D3E05DC0
:10168000AE2F16DEA1EAB0E044CEA091AA01B0913F
:10169000AB018091AC019091AD010895F6DFE8EEC9
:1016A000F3E060E070E07CD3DF01CB01EAE0F0E042
:1016B00060E070E0A8D3E05DAE2F0895E6DFA436C9
:1016C000E0E0BE07E0E08E07E0E09E070895DDDF82
:1016D000E4E6F0E060E070E063D3DF01CB01EAE034
:1016E000F0E060E070E08FD3E05DAE2F0895AFE9E9
:1016F000B0E00FCECADFEAE0F0E060E070E050D387
:10170000DF01CB01EAE0F0E060E070E07CD3E05D77
:10171000AE2FCEDD4ECFAE2FCBCDA091A601B09196
:10172000A7018091A8019091A9010895F6DFE8EE44
:10173000F3E060E070E034D3DF01CB01EAE0F0E0F9
:1017400060E070E060D3E05DAE2F0895E6DFE4E690
:10175000F0E060E070E024D3DF01CB01EAE0F0E0EC
:1017600060E070E050D3E05DD6CFD7DFEAE0F0E094
:1017700060E070E015D3DF01CB01EAE0F0E060E06B
:1017800070E041D3E05DC7CFA0918A01B0918B0199
:1017900080918C0190918D010895AF30E7E2BE07F2
:1017A000E0E08E07E0E09E070895EEDFAF39E6E85F
:1017B000BE07E1E08E07E0E09E070895E5DFA03177
:1017C000E7E2BE07E0E08E07E0E09E070895DCDF79
:1017D000E0E1F7E260E070E0E3D2DF01CB01EAE0B4
:1017E000F0E060E070E00FD3E05DAE2F0895CCDF55
:1017F000E8EEF3E060E070E0D3D2DF01CB01EAE095
:10180000F0E060E070E0FFD2E05DAE2F0895BCDF55
:10181000A436E0E0BE07E0E08E07E0E09E07089512
:10182000B3DFE4E6F0E060E070E0BAD2DF01CB01C4
:10183000EAE0F0E060E070E0E6D2E05DAE2F08950F
:10184000A3DFAA30E0E0BE07E0E08E07E0E09E07FD
:1018500008959ADFEAE0F0E060E070E00895A0D239
:10186000DF01CB01EAE0F0E060E070E0CCD2E05DC7
:10187000AE2F0895C8D2E05D4ECF4BDDD601EAE031
:10188000F0E0089588D2DF01EAE0F0E0AED2E05D5A
:1018900042CFD601EAE0F0E0A8D2E05D3CCFA8EB71
:1018A000B0E037CDEC15FD0508959FD2E05D33CF54
:1018B000EAE0F0E00895A0E021FCA1E0A030089566
:1018C000D9011ACD26DD8DCEE83EA3E0FA07A0E0CF
:1018D0006A07A0E07A070895DF01CB010895E8EEDA
:1018E000F3E060E070E0BBCFF7DFE4E6F0E060E05B
:1018F00070E0089555D2F0DFEAE0F0E060E070E0DB
:10190000B9CFEADFEAE0F0E060E070E00895A0E13E
:10191000B1E0FFCCE8E08E2E08959ADDDF01C8CF5C
:10192000E436A0E0FA07A0E06A07A0E07A0708958D
:10193000AEE0B1E0EEDC77CD2ED2DF01B9DF55D2DB
:10194000E05DAE2F0895BA93AA930895A981BA8154
:101950000895E0E0FCE36CE176EC089579DDEE0FAC
:10196000FF1FEA0FFB1F0895E6DCA0E3E9CC109609
:1019700039F080ED97E00197F1F7A8951197C9F735
:101980000895EE27C398BB9A80EC93E00197F1F796
:10199000BB9885E28A95F1F7B39B08958BEC8A9505
:1019A000F1F7B39BE1E08CE093E00197F1F7089544
:1019B000BB9A85E08A95F1F7BB988DE18A95F1F79E
:1019C0008894B3990894E79585ED8A95F1F7089581
:1019D000E894BB9A85E08A95F1F770FDBB9883E2A5
:1019E0008A95F1F7B39903C070FF03C0089570FFA3
:1019F000089588EC8A95F1F7BB988DE08A95F1F708
:101A00006894089568E0D4DF6A95E9F708957A2F1D
:101A100068E0EE27DDDF26F477956A95D9F7E39540
:101A200008954F935F9311244427012C1124A9DFBB
:101A3000EE2301F1AF93A881EADFAF9151E0501599
:101A400098F4B6DFE7FD08C0B3DFE7FD06C03FD07E
:101A5000892319F4152E01C0ABDF39D0892370E03A
:101A600009F071E0B5DF1EC0A3DFE7FF0BC0A0DF08
:101A7000E7FF05C0E42F5F914F9121960895689488
:101A800037D0EFCF95DFE7FF01C003C0501531F02D
:101A9000152EE8942DD077279BDF04C0689428D0BA
:101AA00071E096DF5395513454F282DFEE1FEE1F42
:101AB000E1701896EC93189743951120D9F259E0EC
:101AC000EC911996EC9318975A95D1F7AECFE52F74
:101AD000EA956E2FE695E695E695FF27EA0FFB1F40
:101AE000808191E0677019F0990F6A95FCCF089595
:101AF000EEDF1EF09095892301C0892B8083089525
:101B0000EE27AA2389F08A2F68E1A881B98198E09D
:101B1000FD917F2F7E27779508F4E627E795F695C8
:101B20009A95B9F78A9599F722960895552342F424
:101B3000503811F4E0FF04C03196691F791F6BF033
:101B400050E8572711F45F9373C05F3F31F0660F81
:101B5000000C57956795752F08955F9300200AF044
:101B600073C06CC050E8192E1522880F991F952755
:101B7000550F879550E8072E0522660F771F7527AA
:101B8000550F67950895689401C0E8945F93F2DF5C
:101B9000703818F07F3F08F44BC056E1571BAAF489
:101BA000519558300EF4593030F0EFEFFFEF6FEFF2
:101BB0007FE777F91AC077275523B9F0EE0FFF1F9B
:101BC000661F771F5A95D1F710C07727583028F035
:101BD000EF2FF62F672F5850F9CF552331F0769518
:101BE0006795F795E7955A95D1F700200AF48ED0BE
:101BF0005F910895689401C0E89430976040704008
:101C0000B1F0002426F0772312F400947FD0172E31
:101C10007EE1112032F07A95EE0FFF1F661F111C36
:101C2000F9CFEF2FF62F612D5F938ADF5F91089533
:101C3000EE27FF27662777275F910895EFEFFFEFE5
:101C40006FE77FEF5F910895EFEFFFEF6FE77FE7BB
:101C50005F9108955F9386DF703851F3903841F3B8
:101C600001240894791F23F41CF300203AF3ECCFED
:101C70000F921F932F933F934F931127222799275A
:101C8000689FA0018F9F302D410D591F6B9F300D14
:101C9000411D591F8E9F27D0BF9F25D06A9F23D0FB
:101CA000BE9F1DD0AF9F1BD0AE9F110D291F391FA6
:101CB000491F591FE32FF42F652F522F4F913F914A
:101CC0002F911F910F9066232AF0550FEE1FFF1FD3
:101CD000661F02C073954BF229DF5F910895100DC6
:101CE000211D391F02C0200D311D491F591F0895A4
:101CF000EA0FFB1F681F791F0895EA1BFB0B680B97
:101D0000790B0895F195E195F0400895F09560956F
:101D10007095E195FF4F6F4F7F4F08956F2F660FBE
:101D2000660B762F0895EE23E1E009F0EE27089583
:101D30007A9F702D6B9F700DF89F700DE99F700D4D
:101D40006A9F602D710DFB9F600D711DE89F600DF6
:101D5000711D8827FA9FF02D610D781FEB9FF00D04
:101D6000611D781FEA9FE02DF10D681F781F08950F
:101D70000024112490E1AA0FBB1F001C111C0E1A95
:101D80001F0A18F40E0E1F1E01C0A1609A9599F744
:101D9000FD01D00108953BD0EBDF0EF4B3DF0895D1
:101DA0003F934F935F93002411244427552730E23B
:101DB000AA0FBB1F881F991F001C111C441F551F11
:101DC0000E1A1F0A460B570B28F40E0E1F1E461F35
:101DD000571F01C0A1603A9559F7FD01BC01D00120
:101DE000CA015F914F913F910895E894B7FF04C0F5
:101DF000A095B09511966894F7FD84DFB9DFFD01D9
:101E00000EF480DF0895CCDFFD01BC010895E89455
:101E1000F7FF02C077DF6894B7FF06C0A095B095C2
:101E2000119600F8039400FA0895ED91FD916D91DB
:101E30007D9108957E936E93FE93EE9308950590A1
:101E4000F491E02D0895A591B4910895182E862F50
:101E5000612D192E972F712D1B2EBF2FF12D1A2EAC
:101E6000AE2FE12D0895129602D0BF011297119660
:101E700002D0FE2F1197E199FECFFF93FFB7F894A0
:101E8000AEBBBFBBE09AEDB3FFBFFF91089507D093
:101E900012960F01FB0103D0F0011297089507D0AD
:101EA0001196EF93EF2F03D0EF9111970895E19BD7
:101EB00002C0A895FCCF9FB7F894AEBBBFBBE09A19
:101EC0008DB3E81719F0EDBBE29AE19A9FBF089530
:101ED0003097604070400895EA17FB07680779075C
:101EE0000895AE17BF078607970708953A932A9378
:101EF0001A930A9308953B812A81198108810895D4
:00000001FF
